:030000000219FDE5
:03000B000200A848
:03002B000201646B
:03005B000202EEB0
:030073000202D4B2
:1000800002030406080C10182030406080040608A3
:100090000C10182030406080A0C000070F1F3F05E3
:1000A000050D050305030302C2AFC0D0C0E0206206
:1000B00017E5256002E473E525F4F58A758B00D217
:1000C00062D0E0D0D0D2AF3285268AC262E526F473
:1000D0006036306803207210758B00D0E0D0D0C23B
:1000E00090C287C291D2AF32C290C287C291206EB5
:1000F0000D20660A7401D5E0FDE57EF45290758B03
:1001000000D0E0D0D0D2AF32758A00C28DD2620169
:10011000FE01B7306805206602D29001B73068054D
:10012000206602D28701B7306805206602D29101AD
:10013000B7D29630680A2066077405D5E0FDD290E4
:1001400001B7D29430680A2066077405D5E0FDD265
:100150008701B7D29530680A2066077405D5E0FD9F
:10016000D29101B7C2AFC2AD53E6EFC0D0C0E0D26A
:10017000D3D2AFC2CEE52A6007207449152A21C523
:100180007800790020742EE580307E01F430E6029C
:1001900078FF53DACF207E0343DA20307E0343DA40
:1001A00010C2D8C271E580307E01F430E60279FFDA
:1001B000C3E89970CB306103752A18207403752A3F
:1001C00018885FD27020740DE52B6004152B21D5A3
:1001D00043DA01C2D82070024137A85F206102C211
:1001E00070207431C3E894F0400374F0F8E8C4540C
:1001F0000F28F87984B703024115C313C31387216D
:10020000200802C313200A06C3C898F8411528F82D
:10021000500374FFF8C3E895685003E568F8882236
:10022000E52D54066011E533C313C31324062522BC
:10023000F52250037522FF852224A824C3E52495C6
:10024000644002A8648825E5697002417BC3E8AA7E
:10025000699A5003E8FAE4F9EAC333FBE56BF45B0F
:1002600029400D256AF8E56A6002156A400B417B5A
:100270000AC3E56A9A5002056A78FF8826C26EC3EF
:10028000E52694F84002D26EC3E52594404002D2A0
:100290006420CF0AD0E0D0D043E610D2AD32C2CF36
:1002A000053A7801E52A6005307402152AC3E55F36
:1002B0009401400575620041CA756300756C00E5E4
:1002C000622401F56250037562FFD0E0D0D043E6AE
:1002D00010D2AD32C2AFC0D053E67FC2607591007C
:1002E000855694855795759104D0D0D2AF32C2AF60
:1002F00053E6EFC2ADC0D0C0E0C0F0D2D3D2AFA8B9
:10030000FBA9FCC2D8307102615553DACF207E03BD
:1003100043DA10307E0343DA20D271E580307E016B
:10032000F420E602612C88278928A18253DACF20A5
:100330007E0343DA20307E0343DA10C2D8C2713024
:100340007402A16E7800E580307E01F430E602A1EF
:100350006E885FA15653DACF207E0343DA20307EC9
:100360000343DA10C271206102812E53DACF207E5E
:100370000343DA10307E0343DA20C2D8D271885AA0
:10038000895BC3E89558F8E99559F97B007E087AAE
:1003900000C3E8948CE994005005755E00812088C4
:1003A0002178A2E6A8216055C3E894C8E9940050DA
:1003B00008E4D2E4FB7A0A61FBC3E89468E994019B
:1003C0005008E4D2E3FB7A0F61FBC3E894D0E994D0
:1003D000025008E4D2E2FB7A1E61FBC3E894A0E974
:1003E00094055008E4D2E1FB7A3C61FBC3E89498A1
:1003F000E994085008E4D2E0FB7A787E00C3E895DF
:100400005CFCE9955DFD30E70AECF42401FCEDF4B9
:100410003400FD755E00C3EC9AED9E5003755E01DD
:10042000885C895D855A58855B597802A156C3E876
:100430009527F8E99528F9307C02A13A307B02A192
:100440003A307A02A1332075028151E9FDE8FC813E
:1004500070E9C313F9E813F8307902A133E9C31343
:10046000F9E813F8307802A133E9C313FDE813FC6F
:0F04700020612CC3EC941CED940240028187EDB7
:10047F00701EC3EC94C850180529E5297002152980
:10048F00C3E529940A5002A16E755F00D270A16E68
:10049F00E529600215297888E6F97400207F08782D
:1004AF0096B90302789EE624FAFEE43400FFC3EC0B
:1004BF009EFCED9FFD9208B90310A208500720760D
:1004CF0009D27681D9307602C276A2085016B903C6
:1004DF000DECF42401FCEDF43400FD0204F378007C
:1004EF007900A13AB90315EC33FCED33FDC3EC945D
:1004FF000AFCED9400FD50047C007D00C3EC94FFDA
:10050F00ED9400400678FF7900A13AEC8575F0A4D0
:10051F00C5F0A2F733F87900400302055678FF794A
:10052F0000020556E9C313F9E813F8307C0EE960B1
:10053F000278FFC3E81338F8E43400F9C3E894FFF6
:10054F00E99400400278FF885FD270206102A16EAB
:10055F00741FF4552F4BF52FC274EB7002D27475C4
:10056F002A18307403752A0A306102A1822074039D
:10057F0053DAFE207403752B06D0F0D0E0D0D0D222
:10058F00AD43E6103279010205B279030205B27963
:10059F000A0205B2791E0205B279640205B279C862
:1005AF000205B27817E4D5E0FDD8FAD9F6227A140D
:1005BF007B780205D97A107B8C0205D97A0D7BB432
:1005CF000205D97A0B7BC80205D97902B27DE4D234
:1005DF0094D5E0FDD287D5E0FDC287D5E0FDC2946A
:1005EF00D5E0FDD290E576D5E0FDC2907496D5E0CA
:1005FF00FDD9D9EAF8D5E0FDD8FBDBCED29422C3E2
:10060F007C007D0075F00005F0EA33FAEB33FB5008
:10061F00F6EB13FBEA13FAC3E9FFE8FEE89AF8E9F1
:10062F009BF95004EFF9EEF8B3EC33FCED33FDD545
:10063F00F0DFEDF9ECF822E889F08A20D2D4F8A99E
:10064F00F07B0030F70B7BFFF42401F8E9F4340062
:10065F00F9E88520F0A4ADF0F8E98520F0A4AFF01B
:10066F00FEED2EF974003FFA7C04C3EA13FAE91386
:10067F00F9E813F8DCF48BF030F70AE8F42401F80A
:10068F00E9F43400F9E889F0C2D4F8A9F02222C3C2
:10069F00E54113F9E54013F8C3E54598F8E54699A8
:1006AF00F9500CC3E89480E994FF40160206D5C3B5
:1006BF00E8947FE9940050030206D5787F79000211
:1006CF0006D5788079FF884A894B22E54A2547F875
:1006DF00E54B3548F9854B20E4300701F43549FAED
:1006EF0030E709C3EA94F04015020713C3EA940FE9
:1006FF00500302071378FF79FF7A0F020713780070
:10070F0079007AF0C3E5249564500AC374019524E7
:10071F00500B020731E54B20E70E020731E54B3056
:10072F00E706884789488A492278A4E6FAC3E54A4A
:10073F0033F8E54B33F9D146E930E70BC3E8948042
:10074F00E994FF4013E16BC3E8947FE994005002F2
:10075F00E16B787F7900E16B788079FFE820E7150E
:10076F00C3E52398F84009C3E894014003020792B8
:10077F007801020792E8F424012523F840030207C9
:10078F009278FF884C2278A5E6FAA848A949D14665
:10079F00E930E70CC3E89401E994FF40160207C65D
:1007AF00C3E894FFE9940050030207C678FF79006D
:1007BF000207C6780179FFE920E715C3E54C98F8E1
:1007CF004009C3E8940140030207ED78010207EDE9
:1007DF00E8F42401254CF840030207ED78FF882444
:1007EF002278FFC26420693D206A12D264C3E541BA
:1007FF00940A4009C3E52594405002C26479A1E7E9
:10080F006023E541601F74FF8541F0848539F03026
:10081F006A0375F005A4F8C5F0600278FFC3E89588
:10082F00675002A867886622C3E5409440E541946B
:10083F0001E5665003140148046002F566220208C0
:10084F00502275E890227883E6FFE5E820ECF7A8C0
:10085F00BDA9BE0573C3E57394084052757300E9D3
:0D086F00FA79A0E76044EA7007E574601BA9
:10087C0002088BC3E895746010E5745006600C1484
:10088C000208970460F9020897E574F574C394673D
:10089C00401B7564C0C394044013756480C39404F6
:1008AC00400B756440C39404400375640075BB0A27
:1008BC0022E564F460020564E573B4070375BB10AC
:1008CC0022743279A687F0A4C5F0A2F733F8C3E8F6
:1008DC0095644002A8648822882488258826886725
:1008EC00227540007541F022C2AF75C820A8CCA972
:1008FC00CDAA3A30CF010A75C824D2AFAB3BAC3C81
:10090C00883B893CC3E89BF8E99C206908F930676F
:10091C000241092166AD3D8A3DF9EA9DFA600478F1
:10092C00FF79FFAE3EAF3F8B3E8C3FC3EC9FFCC3C9
:10093C00E99CF542A83BA93CC3E89EF8E99FF9C3A2
:10094C00E54113FBE54013FAE82AF540E93BF54194
:10095C0050067540FF7541FF21B0AA40AB41AC4039
:10096C00AD417E047F02C3EB940440021E1FC3EB17
:10097C00940840021E1FC3ED13FDEC13FCDEF7C3FD
:10098C00EA9CFAEB9DFBEF6009C3E913F9E813F855
:10099C00DFF7EA28FAEB39FB8A408B4150067BFFE4
:1009AC008B408B41C3EB94025002D2673069047FB9
:1009BC000321DB7892E6FFC3E537948240110FC325
:1009CC00E53794A040010FC3EF940640027F057EEB
:1009DC0004E541C4540FF9E541C454F0F8E540C4B2
:1009EC00540F28F8C3E89EFAE99400FB4009C3EAC7
:1009FC009402EB940050047A02E4FB4155AA40ABFC
:100A0C0041EBC4FEEAC4540F4EFCC3EA9CFAEB94CF
:100A1C0000FBC3E813C313F8EA28FAEB3400FB8A93
:100A2C00408B41C3EB94024002C2677804EBC4FED6
:100A3C007B00EAC4540F4EFAC3EA98FA4005C394FB
:100A4C000250027A027892E6FF30600241558552DC
:100A5C0056855357D26043E680C3E49AF8E49BF979
:100A6C0030670241EFE8FAE9FBD3E913FDE813FC28
:100A7C0088528953C3EF94036038EF20E00DE82CC3
:100A8C00F8E93DF9ECFAEDFB020AAAE828F8E93995
:100A9C00F9C3E82402F8E93400F97AFE7BFFC3EFCE
:100AAC009403400E8A548B55884E894F8C508D512F
:100ABC006123885489558A4E8B4F8C508D513069E7
:100ACC0020C3E53394034019E542A2E713F8E5553A
:100ADC00F4240138400B20E7087554FFF42401F589
:100AEC00556123E8FAD3E813FC8852C3EF940360F2
:100AFC0020EF20E007E82CF8ECFA610FE82824023C
:100B0C00F87AFEC3EF940340088A54884E8C5061E7
:100B1C002388548A4E8C50E56BC3335002646BF5BA
:100B2C006B306002612D753402D26043E680E52D96
:100B3C0054066026A840A941C3E913F9E813F8C28A
:100B4C00AF53E67F759100C3E498F594E499F5955D
:100B5C00759104D26043E680D2AF22D26575440011
:100B6C00752000306B03752040020B86D2657544EE
:100B7C0000752040306B03752000D2AF78012067E0
:100B8C0022E52D54066002C265C3E541940540136D
:100B9C007802940540087803940540027806306981
:100BAC0002780A206019E544601530690AC3E53300
:100BBC0094034003D53406D2AFD26C81577135D231
:100BCC00AF0000C2AF206726E541C3FB940F400283
:100BDC007B0FEB240530730123306A0274282062EA
:100BEC000123F93069027982E58BC39940B505443C
:100BFC00E59B5440B52002814130690A08C3E89452
:100C0C000A40010861AF2065026186C26553E67F28
:100C1C007591003067107594007595FE759104D22E
:100C2C006043E6806186AE40AF41C3E49EF594E438
:100C3C009FF5958128C3E533940250026186306597
:100C4C00026186D802815561AFC26C53E67F759103
:100C5C0000855494855595759104854E56854F574E
:0D0C6C00D26043E680D2AFE52D540660084B
:100C7900206A020533020C91306C0D206B0A206545
:100C89000715811581021514227800306405306535
:100C9900027801E53775F007A4F9E5F028F5F0E9E0
:100CA900A2F013A2F113A2F213F537C394785003FB
:100CB900753778C3E53795384008D266C290C28740
:100CC900C29130600281CB855056855157D260431D
:100CD900E68022207D11C2AF754302D294C296D21A
:100CE900AF759F34020EABC2AF754302D294C29561
:100CF900D2AF759F34020EAB307243207D20C2AF54
:100D0900754303900142757E10C291D295306204F9
:100D1900D287A11FC294D2AF759F35020EABC2AF65
:100D2900754303900142757E10C290D296306204D9
:100D3900D287A13FC294D2AF759F32020EAB207DFC
:100D490017C2AF75430390011DC291306202D28769
:100D5900D2AF759F35020EABC2AF75430390011D2B
:100D6900C290306202D287D2AF759F32020EAB2099
:100D79007D11C2AF754304D296C295D2AF759F3229
:100D8900020EABC2AF754304D295C296D2AF759F1E
:100D990035020EAB307243207D20C2AF75430590FA
:100DA9000131757E40C287D294306204D290A1BBD2
:100DB900C296D2AF759F34020EABC2AF7543059090
:100DC9000153757E20C287D294306204D291A1DB8F
:100DD900C295D2AF759F34020EAB207D17C2AF7595
:100DE9004305900113C287306202D290D2AF759F3A
:100DF90034020EABC2AF754305900127C28730623A
:100E0900EBD291D2AF759F34020EAB207D11C2AFE8
:100E1900754306D295C294D2AF759F35020EABC207
:100E2900AF754306D296C294D2AF759F32020EAB0C
:100E3900307242207D20C2AF754301900153757E07
:100E490020C290D296306204D291C157C295D2AFD6
:100E5900759F32020EABC2AF754301900131757EA9
:100E690040C291D295306204D290C177C296D2AF76
:100E7900759F35C1AB207D16C2AF7543019001271F
:100E8900C290306202D291D2AF759F32C1ABC2AF6C
:100E9900754301900113C291306202D290D2AF75AD
:100EA9009F35C26622900111757E00C290C287C229
:100EB90091D296D294D295C26222788076FF087632
:100EC900FF0876FF0876FF08760308760408760B94
:100ED900087603087601087601788C76010876FF92
:100EE9000876FF0876FF0876FF0876FF087603087C
:100EF90076FF0876FF0876FF0876250876D008760B
:100F0900FA0876FA0876040876FF0876010876006A
:100F190008767A0876FF08760108760108760008CF
:100F29007603227887E6FFC272BF0302D2727888FD
:100F3900E6C394036008C27DE630E102D27DC27E39
:100F49007889E630E102D27EC3EF94026008758E9B
:100F590001D273020F64758E00C273227880E61481
:100F69009000809378A4F67881E6149000809378B5
:100F7900A5F67886E61490008D9378A6F6789CE617
:100F89007538FF75390CB402067538A075390AB47D
:100F9900030675388275390578A3E61490009A938B
:100FA900F569D1AE22227896E6FA7897E6FB788839
:100FB900E6B40305C3EB940EFB307F047A007BFF94
:100FC900C3EB9AFCC3948250027C82757500057547
:100FD900EC8575F0A4C3E5F0947D40F222D27FF14F
:100FE900AF1205A37A007B007C10120599E55F2AF0
:100FF900FA74003BFBDCF37C04C3EB13FBEA13FA42
:10100900DCF7FEC27F120FAF22E5EF20E603752061
:10101900000520903FFFE520146006901DFF146035
:10102900009304600375EF107597DE7597AD7581B0
:10103900C043FF8012059475EF0075A900E5C72428
:101049000420E70DF521E5B120E0068521C743B16C
:1010590001120EAE7580FF75A48075F1C275D4BFFB
:0F10690075907475A57375F27B75D50475A60126
:1010780075E34075E201E4F8F6D8FD756B01120ED0
:10108800C312155678988676753001C2AF1205AD31
:101098001205BD1205A31205C41205A31205CB1231
:1010A80005A312166F1205AD1205AD1205A8C2AF41
:1010B80078FA79FA308607D9FBD8F7021C00120FA4
:1010C8002C120F65120FAE120FAF78988676120E9B
:1010D800AE75885075891275C82475910475D84005
:1010E80075A82275B80275E690759B80759D007588
:1010F800D1BC75BC5875BB0A75E88075B20112057C
:1011080094D2AF12084D53DACF207E0343DA203051
:101118007E0343DA1043DA01C2D8C2711205ADD298
:10112800617B037A0CE55E70077A0CDB030210B66C
:101138001205A32070030210B6C270E55FC39402C3
:1011480040E1E52F541F856160F561B560D5DAD5BA
:10115800C26153DACF207E0343DA20307E0343DABC
:1011680010C2D8C27178A2E67008D274E52F54E094
:10117800F52FC2757529001205A8307409C3E52931
:10118800940A4002D27512059978023074027800E8
:10119800C3E55F9840F0C2AF1205BD1205BD120548
:1011A800BDD2AF1205AD754D007888E6B403024193
:1011B80096120599788CE6C394015003021296E5BD
:1011C80030C394015003021296207435C3E55F942E
:1011D800FF5003021296C2AF1205D2D2AF1205A871
:1011E800C3E55F940150EFC2AF1205BD12059E1210
:1011F80005BDD2AF1205A8C3E55F94FF40E902160A
:10120800F47F05D27F120FAF1205A8C2AFC27F12BA
:101218000FAFAE5FC3E55F947FD2AF407B120594FA
:10122800C2AF1205D2D2AFDFDA120FE6C3EE9405D1
:101238007897F61205AD1215981216777F0AD27FA5
:10124800120FAF1205A8C2AFC27F120FAFAE5FC3B5
:10125800E55F947FD2AF50E4120594C2AF1205BD8A
:1012680012059E1205BDD2AFDFD4120FE6EE24059B
:101278007896F61205AD1215981216A61205A81240
:101288000FAFC3E55F94FF500221D10216F4C3E506
:101298005F954D4003855F4D1205A878017988E771
:1012A800B403027805C3E55F98400221B1C2AF12CA
:1012B80005D21205D21205D2D2AF1205AD75300093
:1012C800E4F531F5320531E531F470390532789AB3
:1012D800E67819146012783214600D787D1460086D
:1012E80078FA146003753200C3E532984017153256
:1012F8007531B478998676C2AF1205D2D2AF789894
:1013080086761205A812059EE52A7005307402013A
:10131800B678012074027806C3E55F9840A77888FC
:10132800E6C3940360031205A8E52A70030210B609
:10133800C2AF120EAEE4F522F523F524F525F52605
:10134800F56AD2AF7885E6C333F568E4F545F54626
:10135800F547F548F549F573F52CF52DF53775730F
:101368000875BB10120594120851E5E820ECFBA89B
:10137800BDA9BEE97001F88874120855757308751F
:10138800BB107887E6FE7602120F2C7887EEF6C23D
:10139800AF7564FF1208CD852264852265852266B3
:1013A800D2AF752201752401752501752601856363
:1013B8006C756D017888E6B40307C27D307602D279
:1013C8007DD268D269753300120E14120E391208D4
:1013D800ED1208F41208ED1208F41208ED0213F5E4
:1013E800C2AF120F2CD2AF75730075BB0A120B78FF
:1013F80012069D120C92120CDC1208F4120B6730C4
:101408006D0312069E2067031207F0306703120867
:1014180037120C92120D011208F4120B78306D037A
:101428001206DA120C92120D781208F4120B6730B9
:101438006D03120738120C92120D9D1208F4120B4C
:1014480078306D03120795120C92120E141208F4DC
:10145800120851120B67120C92120E39120855120B
:0E14680008F4306932206B2F85676485676554
:1014760085636C756D0179187A0CC3E53399400C58
:10148600C269D26A8A357564FF02149FC3E55F9408
:101496000140030213F502151C306A1B206B18E588
:1014A60035147004C26A61E8F535C3E55F940140FE
:1014B600030213F502151C753600C3E5627882989F
:1014C6005054307404E52A604D7888E6B40317203A
:1014D6007D0520760781EC30760281EC206B07D201
:1014E6006B856764813478F0306B05856764782096
:1014F600C3E54198500261F5306B1BC26BC27D306B
:101506007602D27DD26A75351285676461F5053635
:10151600E55F6002A11F753600C2AF120EAE788776
:10152600E6FE7602120F2C7887EEF6E4F522F52316
:10153600F524F525F526F568C268D2AF1205941292
:101546000EAE307409C3E5369405400201B641C8B3
:10155600901A0D78201215DAE520B45A0CA312154C
:10156600DAE520B4A503021578120EC31215980207
:101576001597901A0378807B0A1215DAA308DBF90F
:10158600901A0F788C7B181215DAA308DBF9901ADB
:101596002722C2AF1216191215F3901A00740E12F2
:1015A60015DFA374041215DFA374141215DF901A45
:1015B6000378807B0A1215DEA308DBF9901A0F78F0
:1015C6008C7B181215DEA308DBF912162C12160AEC
:1015D600901A2722E493F622E6438F01538FFD7576
:1015E600EF0275B7A575B7F1F0538FFE22438F0250
:1015F600438F0175EF0275B7A575B7F1901A0DF017
:10160600538FFC22901A0D745AB1DF901A0E74A5EE
:10161600B1DF227A3079D07820901A40B1DAE5200D
:10162600F709A3DAF7227A3079D0901A40E7B1DFCA
:1016360009A3DAF922AB77A878BB01027984BB0249
:10164600027985BB03027986BB04027992BB050247
:101656007987BB060279A3BB0702799CBB0802798E
:1016660088BB09027989E8F7227C051205ADDCFB07
:1016760022C2AF1205BD1205C41205CB1205D21245
:10168600059E1205BD1205C41205CB1205D2120520
:101696009E1205BD1205C41205CB1205D2D2AF2289
:1016A600C2AF1205D21205CB1205C41205BD120532
:1016B6009E1205D21205CB1205C41205BD12059E57
:1016C6001205D21205CB1205C41205BDD2AF22AE49
:1016D60077AF78C2AF1205BD1205BD1205BD120562
:1016E6009EDEF21205D212059EDFF8D2AF22D17726
:1016F600D16FD16F757701757801757900D1D57C79
:1017060005AD5F1205ADC3ED955F70F5C3E55F945A
:1017160001400AC3E55F94FF4032021730D13BB166
:1017260098D177C2AF75EF10D16FDCD50579C3E5D7
:10173600799403500280C6D16F0578E5771490003E
:101746009F93F808C3E57898500280AED16FD16FA9
:101756000577C3E577940A5002809C120EC3B198B0
:07176600C2AF75EF10D16F57
:0319FD00021012C3
:101A00000E0414FFFFFFFF03040B0301015AA5019D
:101A1000FFFFFFFFFF03FFFFFF25D0FAFA04FF01DE
:081A2000007AFF01010003FF41
:101A4000234638355F3341232020202020202020CA
:101A500023424C48454C492346383530232020202A
:101A60002020202020202020202020202020202076
:101C0000C2AFC2D37597DE7597AD7581C075A90057
:101C100043FF80752438752503B1C875EF0275E35D
:101C20004043F14053A4BF75D400D2867DFA7803B7
:101C300079E67C10752200752300901DD57B067512
:101C400024987525013086028145208608D8FBD965
:101C5000F9DCF781B7308608D8FBD9F9DCF781B712
:101C6000B188E493A3C39A6004DDC381B7DBDBB121
:101C70007A6002812E7B08E493FAA3B15BDBF87AE9
:101C800030B15B752200752300B17AEAFCEBFDC32D
:101C9000ED94FE400EB17A8A278B28ED30E0048A5D
:101CA000828B83B17A7AC270D8C3ED94FE601350F0
:101CB000CEBD0023EC60097520007521FF020000F5
:101CC0008100A827A9280809D804D90281D4B17EA7
:101CD000EAF281C80D81A3C3ED94035047EDA2E061
:101CE00092007AC5C3E5829400E583941C5092204B
:101CF0000010438F02438F0175B7A575B7F1F0301F
:101D0000001DA827A9280809438F01538FFDD80477
:101D1000D902A11FE275B7A575B7F1F0A3A10E53C3
:101D20008FFC817F7AC1BD030CE493A3FAB13FDC41
:101D3000F8B137817F8181AA22AB23B15BEBFAEA4C
:101D40006222752608C3E52313F523E52213F52245
:101D500050066323A0632201D526EAB1C8B1C87535
:101D6000260AEAF4200102D286300102C286B1C8F6
:101D7000C3134002C201D526EB22B17EEAFB2086C6
:101D800002A17E308602A183752608AE24AF25C34A
:101D9000EF13FFEE13FEB1CCB1C8C3EA13308602D5
:101DA0004480FA30E703632201C3E52313F523E5FA
:101DB0002213F52250066323A0632201D526D9E51C
:101DC0002265236523F52222AE24AF250E0FDEFE09
:101DD000DFFCD20122424C48656C6934373163F82C
:031DE000500601A9
:00000001FF
